:100000000C94FD040C9444050C9408080C944405CD
:100010000C9444050C9444050C9444050C9444053C
:100020000C9444050C9444050C9444050C94B60DB2
:100030000C94650E0C943F1C0C9444050C944405E0
:100040000C9444050C9444050C9444050C94B31C86
:100050000C9444050C9444050C9444050C944405FC
:100060000C9444050C9444050C9444050C944405EC
:100070000C944405D20EF40EE20FF40EE20F390F89
:100080005C0FE20FB10FC40FE712E712151315133F
:100090007213B013C915C915C913C915CA14CA14E6
:1000A0009D15C915C915B415351F202122232425F6
:1000B00026272D2E742A3A1E2B141A0815171C18E1
:1000C0000C12132F30313B8039041607090A0B0D2F
:1000D0000E0F333432283C7C79781D1B061905112C
:1000E00010363738757D3D7A2C545553494A4B7B31
:1000F0007F8056808080677E5F6061634C4D4E4F8D
:1001000080805780808080805C5D5E624647485179
:100110008080806680808080595A5B294452455097
:100120008080805880808080253032580A002530B9
:1001300032580A004572726F723A20253032580ADE
:1001400000456E640A0073253032583A7225303209
:10015000582000456E61626C6520627265616B3A81
:1001600020004B6579626F6172642049443A202512
:100170003032580A0049424D203437303420636F02
:100180006E7665727465720A00726275663A2066F0
:10019000756C6C0A00523A25303258253032580AB4
:1001A00000533A2530325820004B6579626F6172F6
:1001B000642073746172742E0A0055534220636F79
:1001C0006E666967757265642E0A000D0A696E694C
:1001D000740A003803490042004D00200034003703
:1001E000003000340020006B006500790062006F71
:1001F00000610072006400200063006F006E0076F2
:10020000006500720074006500720000000E037447
:10021000002E006D002E006B002E0000000403096C
:100220000409027400040100A03209040000010363
:10023000010100092111010001224000070581038D
:1002400008000A090401000103010200092111014B
:100250000001224D000705820308000A090402007C
:1002600001030000000921110100012236000705E9
:10027000830308000A0904030002030000000921A7
:100280001101000122220007058403200001070557
:1002900004032000011201100100000008EDFE0718
:1002A000470100010200010631FF0974A10109752F
:1002B000150026FF00952075088102097615002695
:1002C000FF00952075089102C005010980A10185F4
:1002D0000216810026B7001A81002AB70075109512
:1002E000018100C0050C0901A1018503160100264A
:1002F0009C021A01002A9C02751095018100C0051C
:10030000010902A1010901A1000509190129051529
:10031000002501950575018102950175038101058F
:1003200001093009311581257F950275088106097B
:10033000381581257F950175088106050C0A38025C
:100340001581257F950175088106C0C00501090644
:10035000A101050719E029E7150025019508750198
:100360008102950175088101050819012905950586
:10037000750191029501750391010507190029FF87
:10038000150026FF00950675088100C0636F6E7327
:10039000756D65723A20253034580A00737973748C
:1003A000656D3A20253034580A000A00253032584D
:1003B00020006B6579626F6172643A20004C45449D
:1003C0003A20253032580A00253032583A2025305C
:1003D000386225730A00722F63203031323334358E
:1003E00036370A00290A002575002F002575005DA3
:1003F00028002564002000256400200025640020DA
:10040000002564007C0025303258006D6F757365DF
:100410006B6579205B62746E7C7820792076206829
:100420005D287265702F61636C293A205B006D6BEB
:100430005F776865656C5F74696D655F746F5F6D2C
:100440006178203D2025640A006D6B5F77686565E3
:100450006C5F6D61785F7370656564203D20256415
:100460000A006D6B5F74696D655F746F5F6D6178B5
:10047000203D2025640A006D6B5F6D61785F7370AD
:10048000656564203D2025640A006D6B5F696E74AC
:10049000657276616C203D2025640A006D6B5F6497
:1004A000656C6179203D2025640A006D6B5F77687B
:1004B00065656C5F74696D655F746F5F6D617820F1
:1004C0003D2025640A006D6B5F776865656C5F6D24
:1004D00061785F7370656564203D2025640A006D56
:1004E0006B5F74696D655F746F5F6D6178203D202F
:1004F00025640A006D6B5F6D61785F73706565647C
:10050000203D2025640A006D6B5F696E746572760C
:10051000616C203D2025640A006D6B5F64656C6131
:1005200079203D2025640A000A00257500363A200E
:10053000776865656C5F74696D655F746F5F6D6129
:10054000783A20000A00257500353A2077686565FD
:100550006C5F6D61785F73706565643A20000A00B6
:10056000257500343A2074696D655F746F5F6D6145
:10057000783A20000A00257500333A206D61785FD3
:1005800073706565643A20000A00257500323A20D0
:10059000696E74657276616C286D73293A20000A61
:1005A00000257500313A2064656C6179282A313064
:1005B0006D73293A20000A092D2056616C75657308
:1005C000202D0A004D3E004D25643E20003F007363
:1005D00065742064656661756C740A00433E200092
:1005E00077686572652064656C74613A2063757222
:1005F000736F723D25642C20776865656C3D2564BA
:100600000A53656520687474703A2F2F656E2E77D3
:10061000696B6970656469612E6F72672F77696BAA
:10062000692F4D6F7573655F6B6579730A000A09F1
:100630002D204D6F7573656B6579202D0A455343E9
:100640002F713A09717569740A313A0964656C61F0
:1006500079282A31306D73290A323A09696E746536
:100660007276616C286D73290A333A096D61785F7F
:1006700073706565640A343A0974696D655F746FF7
:100680005F6D61780A353A09776865656C5F6D6101
:10069000785F73706565640A363A09776865656CDA
:1006A0005F74696D655F746F5F6D61780A0A703A97
:1006B000097072696E742076616C7565730A643AAC
:1006C000097365742064656661756C74730A75706E
:1006D0003A092B310A646F776E3A092D310A706737
:1006E00075703A092B31300A7067646F776E3A097A
:1006F0002D31300A0A7370656564203D2064656C95
:100700007461202A206D61785F7370656564202AAA
:100710002028726570656174202F2074696D655F93
:10072000746F5F6D6178290A003F004D3E200043E1
:100730003E20004C25640A000A092D20436F6E7389
:100740006F6C65202D0A4553432F713A0971756905
:10075000740A6D3A096D6F7573656B65790A000AE5
:10076000092D204D61676963202D0A643A0964658B
:100770006275670A783A096465627567206D61740D
:100780007269780A6B3A096465627567206B6579EE
:10079000626F6172640A6D3A096465627567206D03
:1007A0006F7573650A763A0976657273696F6E0ABA
:1007B000733A097374617475730A633A09636F6EEF
:1007C000736F6C65206D6F64650A302D343A096C67
:1007D00061796572302D34284631302D4634290A2E
:1007E000506175733A09626F6F746C6F6164657202
:1007F0000A003F0074696D65725F7265616433322F
:1008000028293A202530346C580A006B6579626FCC
:100810006172645F69646C653A2025580A006B65F3
:1008200079626F6172645F70726F746F636F6C3A3C
:100830002025580A00686F73745F6B6579626F6179
:1008400072645F6C65647328293A2025580A000A8F
:10085000092D20537461747573202D0A004743439A
:100860003A20342E392E32204156522D4C494243E3
:100870003A20312E382E3073766E204156525F4129
:100880005243483A2061767233350A004F5054493A
:100890004F4E533A204C554641204D4F5553454BF2
:1008A00045592045585452414B455920434F4E53CA
:1008B0004F4C4520434F4D4D414E44204B45594DE3
:1008C00041505F53454354494F4E20343039360A26
:1008D000004255494C443A20323266366362322037
:1008E0002830303A30373A31362041707220323772
:1008F0002032303137290A005649443A20307846B0
:1009000045454428742E6D2E6B2E29205049443ABB
:10091000203078343730372849424D20343730344E
:10092000206B6579626F61726420636F6E766572A9
:1009300074657229205645523A2030783030303173
:100940000A00444553433A20636F6E766572742003
:1009500049424D2034373034206B6579626F6172C3
:100960006420746F205553420A000A092D205665F1
:100970007273696F6E202D0A000A6D6F7573653A88
:10098000206F66660A000A6D6F7573653A206F6E98
:100990000A000A6B6579626F6172643A206F66665D
:1009A0000A000A6B6579626F6172643A206F6E0AA1
:1009B000000A6D61747269783A206F66660A000AEF
:1009C0006D61747269783A206F6E0A000A6465621C
:1009D00075673A206F6E0A000A64656275673A208F
:1009E0006F66660A000A0A626F6F746C6F616465F5
:1009F000722E2E2E2000433E200011241FBECFEF6A
:100A0000D4E0DEBFCDBF04B603FE27C08091F8015D
:100A10009091F901A091FA01B091FB018730904BC0
:100A2000A740B04BD1F41092F8011092F901109246
:100A3000FA011092FB0114BE84B7877F84BF0FB602
:100A4000F894A8958091600088618093600010926E
:100A500060000FBEE0E0F8E3099511E0A0E0B1E02E
:100A6000E2E9FAE402C005900D92A233B107D9F78A
:100A700021E0A2E3B1E001C01D92A83FB207E1F777
:100A80000E94020B0C9447250C940000FF93EF93F7
:100A9000E0913201F0913301309709F00995EF911F
:100AA000FF910895FC018591803011F0EFDFFBCFBD
:100AB0000895FF27E0E230E247FF0CC0419597FF21
:100AC00009C0EDE26095709580959095611D711D4E
:100AD000811D911D27FF02C0219530E350E2AA2716
:100AE000660F771F881F991FAA1FA41710F0A41B59
:100AF00063955A95A9F7AA3008F0A95FA05DAF9356
:100B0000F395611571058105910541F7ED3211F4F9
:100B1000EF93F395F21718F43F93F395FBCF8F9172
:100B2000B5DFFA95E1F70895E991F9918591803063
:100B300021F0853219F0AADFF9CF089520E0E8947A
:100B400055915532C1F3503311F4689455915A338D
:100B500048F4505390F3220F022E220F220F200D43
:100B6000250FF4CF0EF4219589919991533619F3FD
:100B7000533729F1533559F1BC0188279927E89457
:100B80005C3621F48991999168945591543639F4E1
:100B900046EF7EF077FF0DC08FEF9FEF0AC055370D
:100BA0004AE039F0583540E121F0523642E009F090
:100BB0000895FF93EF937DDFEF91FF91B7CFFF9300
:100BC000EF93FC0181918030B9F360DFFBCFFF939D
:100BD000EF9368DFF1CFDF93CF93CDB7DEB72596E4
:100BE000A3DFCF91DF9108950C942707E82FF0E061
:100BF000EC5CFE4F80810895E4E3F1E080E18E0F2C
:100C000011928E13FDCF0895FF920F931F93CF93F0
:100C1000DF938091DA0181608093DA0185E791E0CA
:100C20000E9452050E94FC052FEF87EA91E62150B1
:100C300080409040E1F700C000000E94FC071F9236
:100C40008F9382E691E09F938F930E94EB0583E55B
:100C500091E00E9452050F900F900F900F908CEF33
:100C60000E943607882339F08FE39CE90197F1F75A
:100C700000C00000F4CFC0E0D0E006E411E08C2F0B
:100C80008068F82E8F2D0E943607882339F08FE375
:100C90009CE90197F1F700C00000F4CF8FE19EE4DA
:100CA0000197F1F700C000000E94FC071F928F938C
:100CB000DF93CF931F930F930E94EB0521960F9024
:100CC0000F900F900F900F900F90CF37D105B9F67E
:100CD0008FEF0E943607882339F08FE39CE9019754
:100CE000F1F700C00000F4CF81E491E0DF91CF91F3
:100CF0001F910F91FF900C945205CF93DF930E94A8
:100D0000FC078F3F09F457C0982F9F779C3778F0E6
:100D10001F928F9384E391E09F938F930E94EB0542
:100D20000E94FC050F900F900F900F9044C090917F
:100D3000DA01C82FC695C695C695D82FD77087FFFC
:100D40001CC090FF0CC01F928F938EE291E09F9386
:100D50008F930E94EB050F900F900F900F90EC2F48
:100D6000EF70F0E0EC5CFE4F81E090E001C0880F96
:100D7000DA95EAF79081892B1BC090FF0CC01F9277
:100D80008F9388E291E09F938F930E94EB050F90E1
:100D90000F900F900F90EC2FF0E0EC5CFE4F81E095
:100DA00090E001C0880FDA95EAF780959081892359
:100DB000808381E001C080E0DF91CF9108950895A4
:100DC0009FB7F8942091480180914901821761F002
:100DD00030E0F901E65BFE4F80812F5F3F4F2F71BE
:100DE00033272093480101C080E09FBF08955198A8
:100DF000599A08955898509A08955098589A089575
:100E00005198599A85E08A95F1F7000089B1869545
:100E1000817008955098589A85E08A95F1F70000FE
:100E200089B181700895CF93DF93C4E6D0E00E942A
:100E30000007811108C0209731F085E08A95F1F70D
:100E400000002197F4CFCE01DF91CF9108950E9449
:100E5000F7060E94FA06E9E6F0E080818C60808364
:100E6000E19AE99A0E94F7060C94FD06BF92CF9290
:100E7000DF92EF92FF920F931F93CF93DF93C82ED1
:100E800010924701E9980E94F7060E94FD065998C2
:100E9000519A0CE211E00E940A0781110AC0011563
:100EA000110549F085E08A95F1F70000015011091C
:100EB000F2CF012B11F480E373C000E010E0D1E029
:100EC000D12CBB24B394C02F0E941307892B11F49B
:100ED000C05C24C0C601002E02C0959587950A9477
:100EE000E2F780FF04C0DB250E94FD0602C00E94DD
:100EF000FA0684E6E82EF12C0E940007882359F0B8
:100F0000E114F10451F085E08A95F1F7000081E0E9
:100F1000E81AF108F1CFEF2821F4C85BC09347012C
:100F20004AC00F5F1F4F0830110569F60E94130772
:100F3000892B11F484E334C0DD2329F00E94FD06DF
:100F400004E610E00CC00E94FA06FACF0115110564
:100F500061F085E08A95F1F70000015011090E94C7
:100F600000078111F3CF012B11F485E319C00E9412
:100F70001307892BF9F20E94FD0604E610E00E9497
:100F80000A07882351F00115110549F085E08A957B
:100F9000F1F7000001501109F2CF012B21F486E393
:100FA0008093470108C00E94F7060E94FD06E19A5F
:100FB000E99A80E017C00E94F7060E94FD06809122
:100FC0004701813360F01F928F9381EA91E09F93F4
:100FD0008F930E94EB050F900F900F900F90E19A66
:100FE000E99A8FEFDF91CF911F910F91FF90EF90D2
:100FF000DF90CF90BF9008952FB7F894909149015A
:10100000809148012FBF98130C94E0068FEF08954C
:101010001F920F920FB60F9211242F933F934F936D
:101020005F936F937F938F939F93AF93BF93CF9370
:10103000DF93EF93FF931092470180914601883030
:10104000F1F030F0893009F05CC0C4E6D0E02EC089
:10105000809145018695809345010E940A07882367
:1010600009F449C08091450180688093450181E081
:1010700090914401911180E0809344013CC00E9412
:101080000A07882339F081E090914401911180E0B2
:101090008093440180914401882399F12CC02097CA
:1010A00081F185E08A95F1F7000021970E940A07F7
:1010B0008111F5CFCD2B29F140914501CFB7F8949F
:1010C0008091490190E09C012F5F3F4F2F713327A2
:1010D00050914801521739F0FC01E65BFE4F408306
:1010E0002093490104C089E891E00E945205CFBFD6
:1010F000109247012AC0809146018F5F809346017C
:101100002AC080914601809347018EEF0E943607E6
:10111000882339F08FE99FE00197F1F700C00000C4
:10112000F4CF809145011F928F93809146011F92C9
:101130008F9385E991E09F938F930E94EB050F9029
:101140000F900F900F900F900F90109246011092F9
:10115000450110924401FF91EF91DF91CF91BF9132
:10116000AF919F918F917F916F915F914F913F913F
:101170002F910F900FBE0F901F90189580917601C0
:1011800008959FB7F89410926D019FBF9091EF0161
:10119000943009F057C09091E9009F703091EC00B5
:1011A000232F217030FD20E8922B24E02093E900CA
:1011B0002091EB0020FF43C02091EE0027FF3FC0AD
:1011C00020916A01222321F02091E80025FF37C0F9
:1011D00010926A0126E03091E80035FD15C030918B
:1011E000EF01343061F53091EB0035FD28C021501E
:1011F00021F481E080936A0122C0EFE9FFE031979A
:10120000F1F700C00000E7CF8093F1008091E80083
:1012100085FD0AC08091E80080FFFCCF8091E80046
:101220008E778093E80006C08FB7F89421E0209372
:101230006D018FBF9F709093E90080E008959F70CB
:101240009093E9008FEF0895CF93DF9300D01F9222
:10125000CDB7DEB79C018091EF01843019F593E0A2
:1012600099833B832A839093E9008FEF9091E80064
:10127000815095FD06C095ED9A95F1F7000081111A
:10128000F5CF8091E80085FF0DC040E050E063E0BD
:1012900070E0CE0101960E94C40B8091E8008E7729
:1012A0008093E8000F900F900F90DF91CF910895F9
:1012B000CF93DF9300D01F92CDB7DEB72091EF011F
:1012C000243021F522E029839B838A8383E0809365
:1012D000E9008FEF9091E800815095FD06C095EDF3
:1012E0009A95F1F700008111F5CF8091E80085FF14
:1012F0000DC040E050E063E070E0CE0101960E9436
:10130000C40B8091E8008E778093E8000F900F90D7
:101310000F90DF91CF9108952091EF012430F1F4E7
:1013200022E02093E9002FEF3091E800215035FDB5
:1013300006C035ED3A95F1F700002111F5CF209167
:10134000E80025FF0BC040E050E065E070E00E943F
:10135000C40B8091E8008E778093E8000895CF93C6
:10136000DF932091EF01243039F521E02093E9004B
:101370002FEF3091E800215035FD06C035ED3A954C
:10138000F1F700002111F5CF2091E80025FF14C0EE
:10139000EC0140E050E068E070E00E94C40B8091F6
:1013A000E8008E778093E80088E0FE01AEE6B1E0C9
:1013B00001900D928A95E1F7DF91CF9108950895FC
:1013C00020916B012F5F822F62E30E940D259923EC
:1013D00019F020936B01089510926B0180916D01BB
:1013E000882371F18091EF01843041F58091E9000B
:1013F0008F702091EC00922F917020FD90E8892B46
:1014000094E09093E9009091EB0090FF14C09091CC
:10141000EE0097FF10C09091E80095FF03C0109276
:10142000F100F9CF9091E80090FF05C09091E8009D
:101430009E779093E8008F708093E90010926D0181
:10144000089542E061EC81E00E94CD0C42E061EC45
:1014500082E00E94CD0C42E061EC83E00E94CD0C62
:1014600042E261EC84E00C94CD0C8091F101833078
:1014700009F453C030F4813071F0823009F48CC02B
:1014800008958A3009F478C08B3009F45EC0893041
:1014900009F09AC020C08091F001813A09F094C00F
:1014A0008091E800877F8093E8008091F40190911B
:1014B000F501892B21F468E08EE691E003C060E03D
:1014C00080E090E070E00E940F0C8091E8008B7744
:1014D0008093E80008958091F001813209F074C092
:1014E0008091F4019091F501892B09F06DC08091F4
:1014F000E800877F8093E8008091E80082FD05C0C6
:101500008091EF018111F8CF5FC08091F10080934D
:1015100076018091E8008B7753C08091F001813A89
:1015200009F052C08091F4019091F501892B09F0E6
:101530004BC08091E800877F8093E8008091E800AD
:1015400080FFFCCF80910A0136C08091F00181328A
:10155000D9F58091F4019091F501892BA9F580913D
:10156000E800877F8093E8000E94020D8091F201DD
:1015700080930A010C94EB158091F001813221F5E2
:101580008091E800877F8093E8000E94020D80919F
:10159000F3018093770108958091F001813AA1F4DD
:1015A0008091E800877F8093E8008091E80080FFC9
:1015B000FCCF809177018093F1008091E8008E77D5
:1015C0008093E8000C94020D089508950895809189
:1015D000760180936C011092760180E00E94DF0614
:1015E0000E94FC050C94EB150C94E70A0E94FE1B6C
:1015F0008091ED01882329F00E94271C81110C9411
:10160000AE0B089584B7877F84BF0FB6F894A89572
:1016100080916000886180936000109260000FBE2E
:1016200090E080E80FB6F894809361009093610099
:101630000FBE81EC98E00E94D31B8BEC91E00E94DE
:1016400052050E94E50A0E94BB100E94530D0E94A1
:10165000A60D8091E20084608093E20078948091EE
:10166000EF018430E1F78AEB91E00E9452050E947D
:10167000BD1080E091E00E94FA0F89EA91E00E949B
:1016800052050E94E60A8091EF01853019F40E940C
:10169000F60AF9CF0E94C110F6CF0E943B1C809140
:1016A0006C018093760108950C944D0B292F3327FC
:1016B00023303105C9F064F42130310581F0223046
:1016C000310509F043C084E790E021E232E042C0F6
:1016D00021323105F1F02232310541F137C082E18A
:1016E00090E025E932E036C099278130910541F03C
:1016F0008230910541F0892B49F5EDE1F2E005C01A
:10170000EDE0F2E002C0E3EDF1E0849190E09F01B2
:1017100021C06430D8F4E62FF0E0EE0FFF1FE15E49
:10172000FE4F2081318189E090E014C0643070F474
:1017300070E0FB01EE0FFF1FE95EFE4F208131815B
:10174000FB01ED5EFE4F808190E004C080E090E000
:1017500020E030E0FA0131832083089584E089BDE0
:1017600086E089BD09B400FEFDCF8091D8008F7D51
:101770008093D8008091E00082608093E0008091A7
:10178000E00081FDFCCF0895CF92DF92EF92FF92AF
:101790000F931F93CF93DF93EC018B016A010E949B
:1017A000210D811133C0C114D10439F0F6018081BB
:1017B0009181081B190BC80FD91FE12CF12C0115C1
:1017C000110519F18091E80085FD16C08091E800AF
:1017D0008E778093E800C114D10449F0F60180812E
:1017E0009181E80EF91EF182E08285E00FC00E942F
:1017F000210D882321F30AC089918093F1000150C3
:101800001109FFEFEF1AFF0ADACF80E0DF91CF91E5
:101810001F910F91FF90EF90DF90CF90089520914E
:10182000F6013091F7012617370748F06115710569
:1018300039F42091E8002E772093E80001C0B90127
:1018400040E06115710591F12091EF01222309F427
:1018500040C0253009F43FC02091E80023FD3DC081
:101860002091E80022FD2FC02091E80020FFE9CF61
:101870002091F20030E0FC01CF016115710559F0B3
:101880002830310540F481918093F1006150710955
:101890002F5F3F4FF1CF41E02830310509F040E0A4
:1018A0002091E8002E772093E800CBCF4111CCCFD8
:1018B0000AC08091EF01882361F0853061F080914A
:1018C000E80083FD0AC08091E80082FFF2CF80E04B
:1018D000089582E0089583E0089581E008952091BD
:1018E000F6013091F7012617370748F061157105A9
:1018F00039F42091E8002E772093E80001C0B90167
:10190000FC0120E06115710579F18091EF018823D8
:1019100009F43DC0853009F43CC08091E80083FDA6
:101920003AC08091E80082FD2CC08091E80080FFE1
:10193000E9CF8091F20090E06115710559F088308F
:10194000910540F424912093F10031966150710982
:101950000196F2CF21E0089709F020E08091E8009D
:101960008E778093E800CECF2111CFCF0AC080912F
:10197000EF01882361F0853061F08091E80083FDFC
:101980000AC08091E80082FFF2CF80E0089582E0F3
:10199000089583E0089581E00895982F953058F5D3
:1019A0009093E900981739F07091EC002091ED00C8
:1019B0005091F00003C0242F762F50E021FF19C072
:1019C0003091EB003E7F3093EB003091ED003D7F96
:1019D0003093ED003091EB0031603093EB00709369
:1019E000EC002093ED005093F0002091EE0027FFD3
:1019F00007C09F5FD3CF8F708093E90081E0089587
:101A000080E008958091F00187FF11C08091E80087
:101A100082FD05C08091EF018111F8CF11C0809146
:101A2000E8008B770BC08091EF01882349F080910B
:101A3000E80080FFF8CF8091E8008E778093E8007F
:101A400008952091E4003091E50095E64091EC0086
:101A5000842F817040FF22C08091E80080FD1CC06F
:101A60008091EF01882391F0853091F08091EB0017
:101A700085FD10C04091E4005091E50042175307E6
:101A800029F39A01915011F784E0089582E00895B6
:101A900083E0089581E0089580E008954091E80092
:101AA00042FFDECF08950E94B00D0E94B30DE0EE1C
:101AB000F0E0808181608083E8EDF0E080818F77C5
:101AC000808319BCE3E6F0E080818160808310921E
:101AD000EE0108950E94B00D0E94B30D8091D800D0
:101AE0008F778093D8008091D80080688093D80049
:101AF0008091D8008F7D8093D80084E089BD86E0F6
:101B000089BD09B400FEFDCF1092EF011092EB01E8
:101B10001092ED011092EC0142E060E080E00E9442
:101B2000CD0C8091E1008E7F8093E1008091E200F6
:101B300081608093E2008091E20088608093E200FF
:101B40008091E0008E7F8093E0000895E3E6F0E06E
:101B500080818E7F808381E08093EE010C946A0DFA
:101B60001092E20008951092E10008951F920F92E2
:101B70000FB60F9211242F933F934F935F936F9360
:101B80007F938F939F93AF93BF93EF93FF93809136
:101B9000E10082FF0BC08091E20082FF07C08091CC
:101BA000E1008B7F8093E1000E94E0098091E100D9
:101BB00080FF19C08091E20080FF15C08091E20093
:101BC0008E7F8093E2008091E20080618093E2004A
:101BD0008091D80080628093D80019BC85E0809302
:101BE000EF010E94F40A8091E10084FF30C08091EF
:101BF000E20084FF2CC084E089BD86E089BD09B481
:101C000000FEFDCF8091D8008F7D8093D800809119
:101C1000E1008F7E8093E1008091E2008F7E8093CF
:101C2000E2008091E20081608093E2008091EB010C
:101C3000882311F084E007C08091E30087FD02C093
:101C400081E001C083E08093EF010E94540B8091FA
:101C5000E10083FF29C08091E20083FF25C08091CD
:101C6000E100877F8093E10082E08093EF01109292
:101C7000EB018091E1008E7F8093E1008091E20092
:101C80008E7F8093E2008091E20080618093E20089
:101C900042E060E080E00E94CD0C8091F00088601E
:101CA0008093F0000E94DF09FF91EF91BF91AF9107
:101CB0009F918F917F916F915F914F913F912F9164
:101CC0000F900FBE0F901F9018951F920F920FB696
:101CD0000F9211242F933F934F935F936F937F93B2
:101CE0008F939F93AF93BF93CF93DF93EF93FF9324
:101CF000C091E900CF708091EC00D82FD17080FDA9
:101D0000D0E81092E9008091F000877F8093F00086
:101D100078940E94A90E1092E9008091F0008860EA
:101D20008093F000CD2BCF70C093E900FF91EF912D
:101D3000DF91CF91BF91AF919F918F917F916F91E3
:101D40005F914F913F912F910F900FBE0F901F9079
:101D500018951F93CF93DF93CDB7DEB7AA970FB631
:101D6000F894DEBF0FBECDBFE0EFF1E088E08E0F4C
:101D70009091F10091938E13FBCF0E94350A8091D0
:101D8000E80083FF1FC18091F0019091F101492F7C
:101D900050E04A30510508F015C1FA01E65CFF4FEA
:101DA0000C942D25803881F0823809F00BC1809188
:101DB000F4018F708093E9008091EB0085FB882708
:101DC00080F91092E90006C08091EC019091ED013C
:101DD000911182609091E800977F9093E800809342
:101DE000F1001092F100C8C0282F2D7F09F0EAC041
:101DF000882319F0823061F0E5C08091F2018130D2
:101E000009F0E0C0933009F080E08093ED012BC031
:101E10008091F201811127C08091F4018F7009F443
:101E2000D1C08093E9002091EB0020FF1CC09330CB
:101E300021F48091EB00806214C09091EB009061DE
:101E40009093EB0021E030E0A90102C0440F551F40
:101E50008A95E2F74093EA001092EA008091EB0045
:101E600088608093EB001092E9008091E800877F02
:101E700086C08111A7C01091F2011F778091E30005
:101E80008078812B8093E3008091E800877F8093A6
:101E9000E8000E94020D8091E80080FFFCCF809155
:101EA000E30080688093E300111102C082E001C06A
:101EB00083E08093EF0186C08058823008F082C0B2
:101EC0008091F2019091F3018C3D53E0950779F5F3
:101ED00083E08A838AE289834FB7F894DE01139600
:101EE00020E03EE051E2E32FF0E050935700E49110
:101EF00020FF03C0E295EF703F5FEF708E2F90E000
:101F0000EA3010F0C79601C0C0968D939D932F5F65
:101F1000243149F74FBF8091E800877F8093E80024
:101F20006AE270E0CE0101960E940F0C14C0AE016F
:101F30004F5F5F4F6091F4010E94560BBC01892BEB
:101F400009F440C09091E800977F9093E800898160
:101F50009A810E946F0C8091E8008B778093E80053
:101F600031C0803879F58091E800877F8093E80060
:101F70008091EB018093F1008091E8008E7780934F
:101F8000E8000E94020D1EC081111CC09091F20158
:101F90009230C0F48091E800877F8093E8009093AE
:101FA000EB010E94020D8091EB01811106C080912E
:101FB000E30087FD02C081E001C084E08093EF016F
:101FC0000E94210A8091E80083FF0AC08091E80006
:101FD000877F8093E8008091EB0080628093EB0024
:101FE000AA960FB6F894DEBF0FBECDBFDF91CF919A
:101FF0001F91089590937D0180937C010895E09155
:102000007C01F0917D01309721F00190F081E02D6D
:10201000099480E00895EF92FF920F931F93CF935E
:10202000DF93E0917C01F0917D013097B1F18C015B
:102030000280F381E02D09958091DA0182FF2DC0A5
:1020400080FF04C082EB93E00E945205E80118E093
:102050008CEAE82E83E0F82E8091DA0180FF0BC035
:1020600088811F928F93FF92EF920E94EB050F9051
:102070000F900F900F90115021961111EDCF80917C
:10208000DA0180FF0AC08AEA93E0DF91CF911F91C5
:102090000F91FF90EF900C945205DF91CF911F911B
:1020A0000F91FF90EF900895E0917C01F0917D01F8
:1020B000309721F00480F581E02D09940895CF93A5
:1020C000DF93EC0180917A0190917B01C817D907C9
:1020D00009F1D0937B01C0937A01E0917C01F091EA
:1020E0007D013097B9F00680F781E02DCE0109958A
:1020F0008091DA0182FF0EC080FF0CC0DF93CF9386
:102100008CE993E09F938F930E94EB050F900F90C3
:102110000F900F90DF91CF910895CF93DF93EC0153
:102120008091780190917901C817D90709F1D0936E
:102130007901C0937801E0917C01F0917D013097A5
:10214000B9F00084F185E02DCE0109958091DA0186
:1021500082FF0EC080FF0CC0DF93CF938CE893E02A
:102160009F938F930E94EB050F900F900F900F900D
:10217000DF91CF9108950C94F4050E94681C0C9493
:1021800004065F926F927F928F929F92AF92BF925E
:10219000CF92DF92EF92FF920F931F93CF93DF9333
:1021A00000D000D01F92CDB7DEB70E947D068FE72A
:1021B000C82E81E0D82E512C88248394912C852D13
:1021C0000E94F605A82EF601E080E82641F453941B
:1021D000FFEFCF1ADF0A80E15812F1CF40C08091A3
:1021E000DA0181FD0E948E1100E010E0F12CB12C8B
:1021F000C701002E02C0959587950A94E2F780FFEB
:1022000028C009835A823401002E02C0660C771C54
:102210000A94E2F793012A213B2181E0232B09F460
:1022200080E08B830E94711C8160782F9D838C835A
:1022300049815A816B818D810E94C41149815A81E3
:102240006B817C818D810E94EB1BF6018081682669
:1022500060820F5F1F4F0830110551F6B8CF8FEF26
:1022600089838A831B820E94711C8160782F9D83E1
:102270008C8349815A816B818D810E94C4110E9497
:10228000EA1B0E943E1F10917E010E94FF0F18174B
:1022900071F10E94FF0F80937E019091DA0192FF0D
:1022A0000EC090FF0CC01F928F938DEB93E09F9315
:1022B0008F930E94EB050F900F900F900F908091DD
:1022C0007E010F900F900F900F900F90DF91CF91A4
:1022D0001F910F91FF90EF90DF90CF90BF90AF9044
:1022E0009F908F907F906F905F900C94FC1B0F904D
:1022F0000F900F900F900F90DF91CF911F910F9142
:10230000FF90EF90DF90CF90BF90AF909F908F9015
:102310007F906F905F9008950C94DF06EF92FF928C
:102320000F931F93CF93DF9386ED93E00E945205A6
:10233000C0E0D0E087E2E82E81E0F82E08EC13E060
:102340008C2F0E94F6050E94D81BFF92EF921F92DD
:102350008F93DF93CF931F930F930E94EB052196EA
:102360008DB79EB708960FB6F8949EBF0FBE8DBF6F
:10237000C031D10529F7DF91CF911F910F91FF90C7
:10238000EF90089508950895CF93DF93CDB7DEB70A
:102390002B970FB6F894DEBF0FBECDBF942F4F839F
:1023A000252F588769877A878B874A855B85452BD8
:1023B00021F02F3F09F59F3FF9F4DE01119686E0E9
:1023C000FD0111928A95E9F785E0FE0137960190AB
:1023D0000D928A95E1F749815A816B817C818D81CB
:1023E0009E810E94A5182B960FB6F894DEBF0FBEF3
:1023F000CDBFDF91CF9108954F81588569857A854A
:102400008B850E94EB1BD9CFCF93882309F465C03D
:10241000C82F8CEF8C0F813A20F080E58C0F8E3224
:1024200048F48C2F0E946A22811157C08C2F0E9481
:10243000341B0CC080E28C0F883058F4C77081E0E8
:1024400001C0880FCA95EAF70E94731BCF910C94C4
:10245000AD1B8BE58C0F833078F4C53A29F0C63A72
:1024600031F083E890E005C081E890E002C082E8A6
:1024700090E0CF910C945F1088E58C0F853168F562
:10248000C83A89F0C93A91F0CA3A99F0CB3AA1F02A
:10249000CC3AA9F0CD3AB1F0CE3AB9F0CF3AC1F08A
:1024A00080E090E017C082EE90E014C089EE90E0EA
:1024B00011C08AEE90E00EC085EB90E00BC086EB79
:1024C00090E008C083EB90E005C084EB90E002C090
:1024D00087EB90E0CF910C948D10CF9108958823D5
:1024E00049F19CEF980F913A20F090E5980F9E32B9
:1024F00018F40E94511B0DC090E2980F983058F4C8
:10250000877091E001C0990F8A95EAF7892F0E94A0
:10251000791B0C94AD1B9BE5980F933020F480E061
:1025200090E00C945F10885A853120F480E090E0B0
:102530000C948D100895882321F00E94731B0C9435
:10254000AD1B0895882321F00E94791B0C94AD1BCC
:102550000895BF92CF92DF92EF92FF920F931F9355
:10256000CF93DF9300D000D000D0CDB7DEB725E009
:10257000FC01DE01119601900D922A95E1F7FC0114
:1025800040813181F280258122952F706381748191
:10259000672B09F4FEC23F3F19F44F3F09F4F9C21B
:1025A0006C0149833A8389819A812E830E94F31AB0
:1025B000182FB92E0E94F21A0E94021AEB2DE295F2
:1025C000EF70F0E0EC5BFF4F2E810C942D258B2DEE
:1025D000807F9B2D9F70092F882311F00295007F2B
:1025E000FF2049F0002309F481C2802F0E94861B3E
:1025F0000E94AD1B7BC2812F0E946F12002309F441
:10260000C8C2802F0E948C1B26960FB6F894DEBF9E
:102610000FBECDBFDF91CF911F910F91FF90EF9033
:10262000DF90CF90BF900C94AD1B8B2D807F9B2DA6
:102630009F70092F803211F00295007F112319F04D
:10264000113009F12AC0FF20B1F0802F222351F16F
:10265000213041F526960FB6F894DEBF0FBECDBFF0
:10266000DF91CF911F910F91FF90EF90DF90CF906E
:10267000BF900C94961B222319F0213009F489C2D3
:102680000E94991B2DC0FF20F1F0263008F081C276
:102690000E94701B802329F023C0FF20F9F0211134
:1026A00016C0802F26960FB6F894DEBF0FBECDBFA2
:1026B000DF91CF911F910F91FF90EF90DF90CF901E
:1026C000BF900C949B12253008F063C209C0F6013C
:1026D000858180FF0BC28F708583E3CF21111BC2E0
:1026E000802F82C12B2D26952695237030E0211551
:1026F000310521F021303105D1F04BC2FF2021F00E
:10270000812F9B2D937002C080E090E026960FB63B
:10271000F894DEBF0FBECDBFDF91CF911F910F9117
:10272000FF90EF90DF90CF90BF900C945F10FF2050
:1027300021F0812F9B2D937002C080E090E02696BF
:102740000FB6F894DEBF0FBECDBFDF91CF911F91C2
:102750000F91FF90EF90DF90CF90BF900C948D1071
:10276000812FFF2019F00E94C41D02C00E942C1E60
:1027700026960FB6F894DEBF0FBECDBFDF91CF9186
:102780001F910F91FF90EF90DF90CF90BF900C942E
:10279000B11E8B2D837009F07BC0F110FAC1812F1F
:1027A000829586958770880F880F912F9F70C92E0C
:1027B000D12CE12CF12C082E04C0CC0CDD1CEE1C1D
:1027C000FF1C0A94D2F714FF12C04FE050E060E003
:1027D00070E004C0440F551F661F771F8A95D2F71B
:1027E000CB01BA01609570958095909503C060E02B
:1027F00070E0CB012B2D269526952370422F50E0BB
:1028000042305105D9F04330510569F16C297D29D9
:102810008E299F294130510551F126960FB6F89423
:10282000DEBF0FBECDBFDF91CF911F910F91FF9003
:10283000EF90DF90CF90BF900C94171A6C297D29F0
:102840008E299F2926960FB6F894DEBF0FBECDBF06
:10285000DF91CF911F910F91FF90EF90DF90CF907C
:10286000BF900C94291A0E94171AC701B601269628
:102870000FB6F894DEBF0FBECDBFDF91CF911F9191
:102880000F91FF90EF90DF90CF90BF900C94051ABE
:10289000FF2019F08B2D817001C08695882309F4E3
:1028A00078C1812F829586958770880F880F912F28
:1028B0009F70C92ED12CE12CF12C082E04C0CC0C19
:1028C000DD1CEE1CFF1C0A94D2F714FF12C04FE06F
:1028D00050E060E070E004C0440F551F661F771F92
:1028E0008A95D2F7CB01BA01609570958095909545
:1028F00003C060E070E0CB012B2D26952695237058
:10290000422F50E042305105D9F04330510569F172
:102910006C297D298E299F294130510551F1269638
:102920000FB6F894DEBF0FBECDBFDF91CF911F91E0
:102930000F91FF90EF90DF90CF90BF900C94CE1A44
:102940006C297D298E299F2926960FB6F894DEBF23
:102950000FBECDBFDF91CF911F910F91FF90EF90F0
:10296000DF90CF90BF900C94E01A0E94CE1AC7015E
:10297000B60126960FB6F894DEBF0FBECDBFDF912D
:10298000CF911F910F91FF90EF90DF90CF90BF906C
:102990000C94BC1A103FC9F128F480E4810F8032F6
:1029A00050F09FC0123F09F461C008F44AC0133FC1
:1029B00009F471C096C0012F00718B2D8F71FF201B
:1029C00051F00E94551A812F002319F08295807FC3
:1029D00069CE8F7067CE0E94761A812F002319F07E
:1029E0008295807F01C08F7026960FB6F894DEBF67
:1029F0000FBECDBFDF91CF911F910F91FF90EF9050
:102A0000DF90CF90BF900C94A212FF20B1F0253040
:102A100008F0BFC08B2D8F7126960FB6F894DEBFDD
:102A20000FBECDBFDF91CF911F910F91FF90EF901F
:102A3000DF90CF90BF900C949B1A263008F0A9C06D
:102A4000E9CFFF20A9F08B2D8F7126960FB6F89451
:102A5000DEBF0FBECDBFDF91CF911F910F91FF90D1
:102A6000EF90DF90CF90BF900C94551AFF2059F350
:102A70008B2D8F7126960FB6F894DEBF0FBECDBF9B
:102A8000DF91CF911F910F91FF90EF90DF90CF904A
:102A9000BF900C94761AFF2099F08B2D8F7126969B
:102AA0000FB6F894DEBF0FBECDBFDF91CF911F915F
:102AB0000F91FF90EF90DF90CF90BF900C94401A51
:102AC00026960FB6F894DEBF0FBECDBFDF91CF9133
:102AD0001F910F91FF90EF90DF90CF90BF900C94DB
:102AE0003B1AFF20A9F0222309F4ADCF812F2696AF
:102AF0000FB6F894DEBF0FBECDBFDF91CF911F910F
:102B00000F91FF90EF90DF90CF90BF900C94041244
:102B1000222309F4ADCF812F26960FB6F894DEBF9D
:102B20000FBECDBFDF91CF911F910F91FF90EF901E
:102B3000DF90CF90BF900C946F124B2D4F70612F90
:102B4000C6010E943A1D26960FB6F894DEBF0FBE4E
:102B5000CDBFDF91CF911F910F91FF90EF90DF904C
:102B6000CF90BF900C944D194B2D4F70612FC60123
:102B700026960FB6F894DEBF0FBECDBFDF91CF9182
:102B80001F910F91FF90EF90DF90CF90BF900C942A
:102B90003D1D26960FB6F894DEBF0FBECDBFDF9168
:102BA000CF911F910F91FF90EF90DF90CF90BF904A
:102BB00008950E94931B0E94621B0E94AD1B0E94FD
:102BC000E51F0E94B11E80E090E00E945F1080E04F
:102BD00090E00C948D100E94831B0C94D9150E94D8
:102BE000F31A292F22952F7030E02C3031054CF448
:102BF0002A303105C4F4225031092230310540F029
:102C000023C02C303105D1F02F303105B9F01CC074
:102C1000853A28F48430B0F4823028F413C090E26E
:102C2000980F983078F0883E30F4803E58F4845005
:102C3000813A50F407C0803F39F404C093FB8827E1
:102C400080F9089581E0089580E00895CF93DF939F
:102C500000D000D01F92CDB7DEB70F900F900F902D
:102C60000F900F90DF91CF910895CF93DF9300D015
:102C700000D000D0CDB7DEB726960FB6F894DEBFF1
:102C80000FBECDBFDF91CF910895CF93DF93C09159
:102C90008F0180919001C817A1F0D0E0CE0166E0CD
:102CA00070E00E94FC24FC01EF56FE4F40815181F0
:102CB00062817381848195810E9435162196C77047
:102CC000E8CFDF91CF9108954091C1015091C201A9
:102CD0006091C3017091C4018091C5019091C601BA
:102CE0000C943516CF93DF938091C60182958F7037
:102CF00009F05CC08091C301882309F457C020917A
:102D00008F01D09190014091C101C091C201E09129
:102D1000C401F091C5012D1709F448C030E0309787
:102D200009F440C0CF3F11F44F3FE1F1C90166E023
:102D300070E00E94FC24DC01AF56BE4F11968C91CE
:102D40001197C8132FC08C9148132CC012968C91E8
:102D50001297811127C013968D919C9114978E170D
:102D60009F0708F401978E1B9F0B883C9105D0F4B8
:102D70008091C6018F7080618093C601C90166E0B1
:102D800070E00E94FC24FC01EA56FE4F90819F7087
:102D90009061908381EC91E00E94A912DF91CF9124
:102DA0000C9445162F5F3F4F2770B5CFDF91CF9121
:102DB0000895BF92CF92DF92EF92FF920F931F93ED
:102DC000CF93DF93CDB7DEB761970FB6F894DEBF30
:102DD0000FBECDBF8C0185E0F801DE011D9601908C
:102DE0000D928A95E1F7D8014C9111962C9111978B
:102DF0001296EC9012971396CD90DC901497509108
:102E0000C1016091C2018091C4019091C5010097F8
:102E100009F46EC16F3F19F45F3F09F469C1B090C6
:102E2000C301BB2009F4C3C03091C601C816D9063E
:102E300028F0F601E81BF90BCF0104C080959095AE
:102E40008C0D9D1DFF24F394883C910588F0F12C96
:102E5000307F09F0CBC07C2DD98AC88A522F6E2DC5
:102E600089890E94261681EC91E00E94A912B4C0C3
:102E7000832F807F09F049C0621314C0541312C01D
:102E8000E11010C03F7030613093C6010E9464169B
:102E900081EC91E00E94A9128091C601D80115969B
:102EA0008C9331C0CD2831F12F3F11F44F3F11F1F8
:102EB000FE2CE1101FC0E0918F0130919001E317CB
:102EC00009F45CC0F0E0CF0166E070E00E94FC24F1
:102ED000DC01AF56BE4F11968C911197281307C095
:102EE0008C91481304C012968C91811103C03196C5
:102EF000E770E5CFFE2CEE2009F416C18091C601E3
:102F000081608093C601F12C0FC1621308C0541375
:102F100006C0E11004C08091C601D801C1C04D8730
:102F20002E878D859E850E94EF158823E1F1EE2086
:102F3000D1F12091C601822F82958F7090E0029787
:102F400074F08091C1019091C20198878F83198696
:102F5000DB86CA862C87CE0107960E94A91286E0DE
:102F6000F801A1ECB1E001900D928A95E1F70E9481
:102F700072160E946416FF24F394D6C04D872E87E4
:102F80008D859E850E94F31A292F22952F7030E09F
:102F9000223031050CF0BCC09F7009F0B6C0805ED5
:102FA000883008F4C1C0C8010E94A912E4CFC81635
:102FB000D90608F453C0F601E81BF90BCF01883C91
:102FC000910508F450C0F12C7C2DD98AC88A522F63
:102FD0006E2D89890E942616E1ECF1E086E0DF0182
:102FE0001D928A95E9F70E9464169EC0621314C070
:102FF000541312C0E11010C08091C601F8018583FE
:10300000C8010E94A91286E0E1ECF1E0DF011D9207
:103010008A95E9F7FB2C88C04D872E878D859E8584
:103020000E94EF15882309F4BECFEE2009F4BBCF30
:103030002091C601822F82958F7090E002970CF448
:103040008ECF8091C1019091C2019A8389831B82A6
:10305000DD82CC822E83CE0101967FCF8095909524
:103060008C0D9D1DACCFFE2CEE2009F49CCF62137D
:103070002EC054132CC02091C60120FD1FC0822FEA
:1030800082958F70D9F0D80115962C9315978F30B3
:1030900049F08F5F982F9295907F822F8F70892BA8
:1030A00015968C93C8010E94A91286E0F801A1EC44
:1030B000B1E001900D928A95E1F795CF86E0F80195
:1030C000A1ECB1E001900D928A95E1F72DC04D87FA
:1030D0002E878D859E850E94EF15811140CF8091AE
:1030E000C60181608093C601C8010E94A9121CC05C
:1030F000EE2009F458CF4D872E878D859E850E943E
:10310000EF15882309F44FCF2ACF811148CF0CC087
:10311000243031050CF047CF9F7009F440CFF801FF
:103120009581907F09F03BCF8F2D61960FB6F89473
:10313000DEBF0FBECDBFDF91CF911F910F91FF90EA
:10314000EF90DF90CF90BF900895CF93DF93CDB7EE
:10315000DEB72C970FB6F894DEBF0FBECDBF4F83FE
:10316000588769877A878B879C87CE0107960E944C
:10317000D916882371F08F8198852A853B85232B6A
:1031800009F43FC09F3F09F068C08F3F09F065C058
:1031900038C086E0FE013796DE01119601900D924F
:1031A0008A95E1F76F817885EA85FB85309749F14B
:1031B0007F3F11F46F3F29F18091900190E09C01D5
:1031C0002F5F3F4F2770332740918F0150E0241726
:1031D000350709F44BC069837A83FD83EC8366E08D
:1031E00070E00E94FC24DC01AF56BE4F96E0FE0169
:1031F000319601900D929A95E1F7209390010E94EB
:10320000451680918F01909190018917E9F190E026
:1032100066E070E00E94FC248F569E4F0E94D916F3
:10322000882391F180918F0190E066E070E00E9428
:10323000FC24FC01EF56FE4F408151816281738175
:10324000848195810E94351680918F0190E00196CE
:103250008770992780938F01D4CF4F8158856985D6
:103260007A858B859C850E943516CBCF0E94EB1505
:103270001092900110928F01E1ECF1E086E0DF0105
:103280001D928A95E9F7BDCF2C960FB6F894DEBF54
:103290000FBECDBFDF91CF910895DF92EF92FF92E5
:1032A0000F931F93CF93DF93FC01892B09F48AC0FE
:1032B000E12CF12CDD24D394EF0121968491853704
:1032C00009F461C058F4843708F04EC0843008F027
:1032D0006AC08130D1F0823071F174C0883709F44E
:1032E0005DC050F4863709F455C0873709F06AC0CD
:1032F0008E2D0E94801B54C09CE7980F903708F0D9
:1033000061C08F770E946F1250C08F010E5F1F4FF8
:10331000FE01849190E2980F983050F48770FD2D53
:1033200001C0FF0F8A95EAF78F2F0E94861B14C0F9
:103330000E94041213C08F010E5F1F4FFE01C49143
:1033400080E28C0F883060F4C7708D2D01C0880F2B
:10335000CA95EAF70E948C1B0E94AD1BE80125C0AC
:103360008C2F0E946F12FACF9F012E5F3F4FFE01FC
:10337000C491CC2369F08FE99FE00197F1F700C079
:103380000000C150F6CF9F012E5F3F4FFE01F49029
:10339000E9010BC00E94701BE82E07C00E94831B2E
:1033A0000E94AD1B02C00E9404128F2D882341F0A1
:1033B000EFE9FFE03197F1F700C000008150F6CF50
:1033C000FE017ACFDF91CF911F910F91FF90EF9087
:1033D000DF9008956093CB017093CC018093CD0171
:1033E0009093CE010E94FA1B0C94D9156093C701EB
:1033F0007093C8018093C9019093CA010E94FB1B7E
:103400000C94D91508950C94EA190F931F93009109
:10341000CB011091CC012091CD013091CE01602BD8
:10342000712B822B932B1F910F910C94EA190F9300
:103430001F930091CB011091CC012091CD013091CF
:10344000CE0160237123822393231F910F910C944B
:10345000EA190F931F930091CB011091CC01209199
:10346000CD013091CE0160277127822793271F91CC
:103470000F910C94EA1960E070E0CB010C94F619FE
:103480000F931F9341E050E060E070E08A019B01E0
:1034900004C0000F111F221F331F8A95D2F7C901E4
:1034A000B8011F910F910C94F6190F931F9341E0EF
:1034B00050E060E070E004C0440F551F661F771FA6
:1034C0008A95D2F78091C7019091C801A091C90156
:1034D000B091CA018A019B01082B192B2A2B3B2B87
:1034E000C901B8011F910F910C94F6190F931F9306
:1034F00041E050E060E070E004C0440F551F661FDB
:10350000771F8A95D2F74095509560957095809178
:10351000C7019091C801A091C901B091CA018A0167
:103520009B01082319232A233B23C901B8011F91BA
:103530000F910C94F6190F931F9341E050E060E057
:1035400070E004C0440F551F661F771F8A95D2F79D
:103550008091C7019091C801A091C901B091CA01A1
:103560008A019B01082719272A273B27C901B8018F
:103570001F910F910C94F6190F931F930091C7019F
:103580001091C8012091C9013091CA01602B712BA3
:10359000822B932B1F910F910C94F6190F931F936D
:1035A0000091C7011091C8012091C9013091CA0151
:1035B00060237123822393231F910F910C94F6199A
:1035C0000F931F930091C7011091C8012091C90169
:1035D0003091CA0160277127822793271F910F918D
:1035E0000C94F6190895CF92DF92EF92FF920F9309
:1035F0001F93CF93DF938C01C090CB01D090CC016F
:10360000E090CD01F090CE014091C7015091C801EA
:103610006091C9017091CA01C42AD52AE62AF72A05
:10362000CFE1D0E0D701C6010C2E04C0B695A79516
:10363000979587950A94D2F780FF07C0B8018C2F21
:103640000E940B1D8130910531F4219758F7B80184
:1036500080E00E940B1DDF91CF911F910F91FF9091
:10366000EF90DF90CF90089520910B0130910C01E5
:10367000F90132969FEF40E05191581789F09F3F32
:1036800019F4511101C0942F4F5F4630A9F79F3FA5
:1036900039F0F901E90FF11D97FDFA95828308953C
:1036A000089520910B0130910C01F9013296285FA9
:1036B0003F4F9081981301C010823196E217F307B3
:1036C000C1F7089581E090E0E0910B01F0910C01C9
:1036D000E80FF91F1082019688309105A9F7089527
:1036E0008091D90108959091D901892B8093D901B6
:1036F000089580959091D90189238093D9010895E7
:103700008093D90108951092D90108959091D8011C
:10371000892B8093D801089580959091D8018923B1
:103720008093D80108951092D80108958093CF0115
:1037300008951092CF01089580910B0190910C0192
:10374000FC0131969C01285F3F4F80E091919111DF
:103750008F5FE217F307D1F70895E0910B01F09125
:103760000C018091D9018083E0910B01F0910C0153
:1037700090818091D801892B80838091CF0188230B
:1037800061F0E0910B01F0910C019081892B808315
:103790000E949C1B81111092CF0180910B0190918E
:1037A0000C010C940B109093330180933201089517
:1037B0008295982F9C7C292F26952695982F937378
:1037C000990F990F922B892F8A7A86959575990F63
:1037D000892B08950895CF93DF9300D000D01F92D6
:1037E000CDB7DEB70F900F900F900F900F90DF9135
:1037F000CF910895089508950C948C118091EF0154
:10380000843021F11092DB0120E488E190E00FB6D2
:10381000F894A895809360000FBE2093600083B752
:10382000817F846083BF83B7816083BF78948895EC
:1038300083B78E7F83BF0FB6F894A8958091600000
:10384000886180936000109260000FBE0895CF934E
:103850000E94C2110E947D060E94C311C0E08C2FFD
:103860000E94F605811104C0CF5FC031C1F701C0CD
:1038700081E0CF9108950E94FC050C94EB151F92F6
:103880000F920FB60F9211248F939F93AF93BF9314
:103890008091DB01811113C08091DC019091DD01E9
:1038A000A091DE01B091DF014196A11DB11D809371
:1038B000DC019093DD01A093DE01B093DF01BF91A5
:1038C000AF919F918F910F900FBE0F901F90189501
:1038D00082E084BD93E095BD9AEF97BD80936E0022
:1038E00008952FB7F8948091DC019091DD01A091AB
:1038F000DE01B091DF012FBF08952FB7F8946091DA
:10390000DC017091DD018091DE019091DF012FBF1C
:103910000895CF92DF92EF92FF920F931F932FB7EC
:10392000F8944091DC015091DD016091DE017091CD
:10393000DF012FBF6A017B01EE24FF248C0120E010
:1039400030E0C016D106E206F30610F441505109EA
:103950009A01281B390BC9011F910F91FF90EF901D
:10396000DF90CF9008951F920F920FB60F921124FF
:103970008F939F93AF93BF938091DC019091DD0172
:10398000A091DE01B091DF010196A11DB11D8093D0
:10399000DC019093DD01A093DE01B093DF01BF91C4
:1039A000AF919F918F910F900FBE0F901F90189520
:1039B0000E94530DF8942FEF87EA91E62150804042
:1039C0009040E1F700C0000087E090EBDC018093BD
:1039D000F8019093F901A093FA01B093FB019CE0E8
:1039E00088E10FB6F894A895809360000FBE90937D
:1039F0006000FFCFE92FF0E093E0EE0FFF1F9A95F4
:103A0000E1F7E80FF11DE855FF4F9491892F8F7072
:103A100092959F700895CF93C82FCB010E94FA1CF6
:103A2000492F90E0242F30E054E0220F331F5A95A5
:103A3000E1F7282B392B2038310519F480E090E08C
:103A400017C0EC2FF0E023E0EE0FFF1F2A95E1F7FF
:103A50004770E40FF11D34E0EE0FFF1F3A95E1F7D8
:103A6000E80FF91FEE0FFF1FE050F8498591949180
:103A7000CF91089580E090E0089508958091E2014B
:103A800080FF0CC08091100190E065E070E00E9422
:103A9000FC2495958795959587952EC081FF0AC042
:103AA0008091100190E065E070E00E94FC24959503
:103AB000879522C082FF08C08091100190E065E0E8
:103AC00070E00E94FC2418C02091E3012223D1F071
:103AD00030910F01231780F78091100190E065E08D
:103AE00070E00E94FC24622F70E00E94FC24632F8F
:103AF00070E00E941925CB018038910530F40097C1
:103B000031F0089585E090E008958FE7089581E011
:103B100008958091E20180FF08C060910E0170E07D
:103B2000759567957595679523C081FF06C060916F
:103B30000E0170E0759567951BC082FF04C060910F
:103B40000E0170E012C06091E3016623D1F0209174
:103B50000D016217A0F780910E0170E090E00E94C5
:103B6000FC24622F70E00E9419256038710528F44A
:103B70006115710521F0862F08958FE7089581E082
:103B8000089561E070E0F4CF803F21F40E943E1D73
:103B9000819504C0813F29F40E943E1D8093E60177
:103BA0000895823F21F40E943E1D819504C0833F09
:103BB00029F40E943E1D8093E5010895893F19F480
:103BC0000E94891D05C08A3F31F40E94891D81959C
:103BD0008093E70108958B3F21F40E94891D819510
:103BE00004C08C3F29F40E94891D8093E801089548
:103BF000843F21F48091E401816017C0853F21F466
:103C00008091E401826011C0863F21F48091E4013B
:103C100084600BC0873F21F48091E401886005C077
:103C2000883F31F48091E40180618093E40108953C
:103C30008D3F21F48091E20181600BC08E3F21F421
:103C40008091E201826005C08F3F29F48091E201FA
:103C500084608093E2010895803F39F48091E60109
:103C600087FF6CC01092E60169C0813F29F4809102
:103C7000E6011816BCF362C09091E501823F29F479
:103C800097FF5CC01092E50159C0833F19F41916E3
:103C9000CCF354C0893F41F48091E70118160CF031
:103CA0004DC01092E7014AC08A3F29F48091E70194
:103CB00087FF44C0F6CF8B3F39F48091E80187FF3E
:103CC0003DC01092E8013AC08C3F29F48091E80190
:103CD0001816BCF333C0843F21F48091E4018E7F39
:103CE00017C0853F21F48091E4018D7F11C0863F8C
:103CF00021F48091E4018B7F0BC0873F21F48091F8
:103D0000E401877F05C0883F31F48091E4018F7E14
:103D10008093E40113C08D3F21F48091E2018E7FF6
:103D20000BC08E3F21F48091E2018D7F05C08F3F53
:103D300029F48091E2018B7F8093E2018091E5017B
:103D400081110EC08091E60181110AC08091E701C6
:103D5000811106C08091E801811102C01092E30137
:103D600008958091DA0183FF7EC08BE094E00E9489
:103D700052058091E4011F928F9386E094E09F9317
:103D80008F930E94EB0584E094E00E94520580919D
:103D9000E501282F082E000C330B3F938F9381E011
:103DA00094E09F938F930E94EB058FEF93E00E9426
:103DB00052058091E601282F082E000C330B3F930B
:103DC0008F938CEF93E09F938F930E94EB058AEF84
:103DD00093E00E9452058091E701282F082E000CE5
:103DE000330B3F938F9387EF93E09F938F930E94C2
:103DF000EB0585EF93E00E9452058091E801282FA2
:103E0000082E000C330B3F938F9382EF93E09F9328
:103E10008F930E94EB058FEE93E00E9452058091F4
:103E2000E3011F928F938CEE93E09F938F930E94F8
:103E3000EB058AEE93E00E9452058091E2011F9209
:103E40008F9387EE93E09F938F930E94EB0584EE10
:103E500093E00E9452058DB79EB74C960FB6F8942A
:103E60009EBF0FBE8DBF84EE91E00E9454100E9451
:103E7000711C9093E1018093E00108951F93CF930B
:103E8000DF938091E0019091E1010E94891CFC0187
:103E90002091E301222329F090911101892F90E0D4
:103EA00007C08091120190E06AE070E00E94FC245B
:103EB000E817F90708F485C08091E501C091E60193
:103EC000D091E7011091E801811107C0C11175C0BF
:103ED000D11173C0111171C074C02F3F19F02F5F41
:103EE0002093E301181624F40E943E1D8093E501FF
:103EF0008091E50187FF05C00E943E1D819580935A
:103F0000E5011C1624F40E943E1D8093E601809179
:103F1000E60187FF05C00E943E1D81958093E60162
:103F20006091E501662331F1C091E601CC2311F1E6
:103F3000062E000C770B880B990B0E94FB2323E3C2
:103F400033E343E35FE30E945F240E94C323609353
:103F5000E5016C2FCC0F770B880B990B0E94FB238C
:103F600023E333E343E35FE30E945F240E94C32320
:103F70006093E6011D1624F40E94891D8093E701D9
:103F80008091E70187FF05C00E94891D819580937C
:103F9000E701111624F40E94891D8093E8018091A5
:103FA000E80187FF05C00E94891D81958093E80183
:103FB000DF91CF911F910C94B11E2F3F09F08FCF4D
:103FC00097CFDF91CF911F910895E4EEF1E085E066
:103FD000DF011D928A95E9F71092E3011092E20148
:103FE00008958EE296E00E9452051F9281E08F9321
:103FF0001F9285E08F9380EE95E09F938F930E94B0
:10400000EB050F900F900F900F900F900F90089569
:104010008330E9F128F4813061F0823009F10895AC
:10402000853009F462C008F449C0863009F474C0D0
:10403000089580911201262F30E0280F311D2F3F67
:10404000310524F4680F6093120103C08FEF809351
:104050001201809112011F928F9389E195E072C045
:1040600080911101262F30E0280F311D2F3F31059F
:1040700024F4680F6093110103C08FEF8093110146
:10408000809111011F928F9387E095E05BC0809132
:104090001001262F30E0280F311D2F3F310524F469
:1040A000680F6093100103C08FEF8093100180911F
:1040B00010011F928F9384EF94E044C080910F0110
:1040C000262F30E0280F311D2F3F310524F4680FD3
:1040D00060930F0103C08FEF80930F0180910F0158
:1040E0001F928F938FED94E02DC080910E01262FAB
:1040F00030E0280F311D2F3F310524F4680F609305
:104100000E0103C08FEF80930E0180910E011F926C
:104110008F9386EC94E016C080910D01262F30E03D
:10412000280F311D2F3F310524F4680F60930D01D6
:1041300003C08FEF80930D0180910D011F928F932B
:104140008BEA94E09F938F930E94EB050F900F9062
:104150000F900F900895833081F128F4813059F049
:104160008230D1F00895853009F449C0B8F1863025
:1041700009F456C0089580911201681720F4861B37
:104180008093120102C010921201809112011F92BD
:104190008F938CE994E054C080911101681720F44A
:1041A000861B8093110102C01092110180911101B0
:1041B0001F928F938AE894E043C0809110016817A2
:1041C00020F4861B8093100102C010921001809190
:1041D00010011F928F9387E794E032C080910F0106
:1041E000681720F4861B80930F0102C010920F0104
:1041F00080910F011F928F9382E694E021C08091FD
:104200000E01681720F4861B80930E0102C01092E5
:104210000E0180910E011F928F9389E494E010C0EB
:1042200080910D01681720F4861B80930D0102C058
:1042300010920D0180910D011F928F938EE294E0F8
:104240009F938F930E94EB050F900F900F900F900C
:104250000895CF93C82F1F928F9383E397E09F9386
:104260008F930E94EB0581E090E0A0E0B0E0BC01FC
:10427000CD0104C0660F771F881F991FCA95D2F71A
:104280000E94031A0F900F900F900F90CF910C94F3
:10429000EB15CF93873288F58E3108F00BC18E3045
:1042A00009F487C0D8F4873009F460C08B3009F472
:1042B0004FC0863009F002C18091DA01817F8E7F84
:1042C0008093DA0188E397E00E94520586EF99E037
:1042D0000E94520581E08093EA0146C0863109F4CC
:1042E000B0C020F4803109F47AC0E8C0893109F403
:1042F00091C08B3109F449C0E1C0883349F150F4D1
:10430000893209F4D5C0853309F4D2C0873209F067
:10431000D5C0CEC0833409F4CBC028F48A3308F466
:10432000CDC08953C8C0883409F0C8C00E94EB15BD
:1043300085EE99E00E9452052FEF83ED90E3215026
:1043400080409040E1F700C000000E94D81C0CC0E3
:104350008FE597E041C08CEC99E00E945205809176
:10436000DA0181608093DA01C1E0ADC08091DA01A9
:10437000C82FC17080FFEFCF88ED99E00E945205F1
:104380008091DA01817F8E7F3FC09091DA0191FBAD
:10439000CC27C0F981E0C827892FC0FB81F9809321
:1043A000DA01CC2319F08FEB99E029C081EB99E079
:1043B00013C09091DA0192FBCC27C0F981E0C827A5
:1043C000892FC0FB82F98093DA01CC2319F082EAAD
:1043D00099E015C082E999E00E945205C5CF9091FD
:1043E000DA0193FBCC27C0F981E0C827892FC0FBF5
:1043F00083F98093DA01CC2351F086E899E00E949A
:1044000052058091DA0181608093DA015CC089E70E
:1044100099E0E2CF8AE699E00E94520582E499E0B1
:104420000E94520588EF98E00E94520581ED98E0C5
:104430000E9452058CE898E00E9452058DE598E0B4
:10444000CBCF8FE498E00E9452050E94FF0F1F928D
:104450008F9385E398E09F938F930E94EB05809163
:104460000A011F928F938EE198E09F938F930E9491
:10447000EB05809177011F928F938BE098E09F93DB
:104480008F930E94EB050E947D1C9F938F937F93D7
:104490006F9384EF97E09F938F930E94EB058DB706
:1044A0009EB742960FB6F8949EBF0FBE8DBF5CCFED
:1044B00080E001C08D510E94292156CF82EF97E004
:1044C0000E945205C0E08C2FCF91089580E008959E
:1044D00080E00895CF93C82F8091EA01813081F068
:1044E00020F0823009F44FC046C1E0910B01F091F9
:1044F0000C018081813169F0823209F03EC109C02E
:10450000E0910B01F0910C018081813111F0823238
:1045100061F48C2F0E946622811104C08C2F0E94AE
:1045200049212FC081E090E02CC08C2F0E9468228E
:10453000811126C0C431E1F070F4CB3081F0C0317C
:10454000D1F40E94F11F8BE297E00E94520582E0B5
:104550008093EA0115C0C93259F0C83361F488E389
:1045600097E00E9452058FE297E00E94520508C032
:104570001092EA0104C189E297E00E945205FFC04F
:1045800081E08170FEC0C43228F5CE3108F0C1C090
:10459000CB30A1F1D0F4C73009F0D3C08EE18093C5
:1045A000120182E3809311018AE08093100184E17B
:1045B00080930F0188E080930E0188E280930D01C3
:1045C0008FEC95E00E945205BFC0C33149F1C43160
:1045D000C1F0B7C0CB3409F4A9C028F4C93289F0BE
:1045E000C83361F0AEC0C13509F49EC0C23509F4CC
:1045F00099C0CE3409F0A5C06AE09EC00E94F11FA8
:10460000A3C08091E901882319F01092E9019CC0B0
:104610008CED95E00E94520581E08093EA01B1C0E3
:1046200086EB95E00E94520584EA95E00E945205CF
:10463000809112011F928F9381EA95E09F938F934F
:104640000E94EB058FE995E00E9452058DE895E008
:104650000E945205809111011F928F938AE895E084
:104660009F938F930E94EB0588E895E00E94520586
:1046700089E795E00E945205809110011F928F9367
:1046800086E795E09F938F930E94EB0584E795E082
:104690000E94520583E695E00E94520580910F0129
:1046A0001F928F9380E695E09F938F930E94EB0576
:1046B0008EE595E00E94520589E495E00E9452053E
:1046C00080910E011F928F9386E495E09F938F93C4
:1046D0000E94EB0584E495E00E9452058DE295E08E
:1046E0000E94520580910D011F928F938AE295E0FE
:1046F0009F938F930E94EB0588E295E00E945205FC
:104700008DB79EB748960FB6F8949EBF0FBE8DBF6B
:104710001BC0CE51EC2FF0E0E85DFE4F808180930E
:10472000E90112C061E003C061E006C06AE0809167
:10473000E9010E94082008C08091E9010E94AB2095
:1047400003C08DEC95E013C08091E901882369F0E6
:104750001F928F9387EC95E09F938F930E94EB05B8
:104760000F900F900F900F9004C084EC95E00E9482
:10477000520581E006C01092EA0180E002C080E0AC
:1047800000CFCF9108950E94CA236894B1110C9470
:10479000592408950E943E2488F09F5798F0B92F1D
:1047A0009927B751B0F0E1F0660F771F881F991F66
:1047B0001AF0BA95C9F714C0B13091F00E9458248C
:1047C000B1E008950C945824672F782F8827B85F9C
:1047D00039F0B93FCCF3869577956795B395D9F7BE
:1047E0003EF490958095709561957F4F8F4F9F4FC8
:1047F0000895E89409C097FB3EF4909580957095D4
:1048000061957F4F8F4F9F4F9923A9F0F92F96E91C
:10481000BB279395F695879577956795B795F11191
:10482000F8CFFAF4BB0F11F460FF1BC06F5F7F4F2E
:104830008F4F9F4F16C0882311F096E911C0772340
:1048400021F09EE8872F762F05C0662371F096E849
:10485000862F70E060E02AF09A95660F771F881F18
:10486000DAF7880F9695879597F9089557FD905830
:10487000440F551F59F05F3F71F04795880F97FB24
:10488000991F61F09F3F79F08795089512161306DE
:104890001406551FF2CF4695F1DF08C0161617060D
:1048A0001806991FF1CF8695710561050894089542
:1048B000E894BB2766277727CB0197F908950E94D4
:1048C00071240C94EB240E94DD2438F00E94E4242F
:1048D00020F0952311F00C94D4240C94DA240C9439
:1048E00059240E94362478F39923C9F35523B9F348
:1048F000950F50E0551FAA27EE27FF27BB2700245E
:104900000894679520F4E20FF31FB41F0A1E220FCC
:10491000331F441FAA1F6695A9F7779530F4F30F4C
:10492000B41F0A1E121E08F46395330F441FAA1FFA
:10493000221F769599F7879520F4B40F0A1E121E50
:10494000631F440FAA1F221F331F8695A9F7862FC6
:10495000712D602D11249F5750409AF0F1F088235B
:104960004AF0EE0FFF1FBB1F661F771F881F915075
:104970005040A9F79E3F510580F00C94D4240C942C
:1049800059245F3FE4F3983ED4F386957795679575
:10499000B795F795E7959F5FC1F7FE2B880F911D9F
:1049A0009695879597F9089597F99F6780E870E045
:1049B00060E008959FEF80EC089500240A94161695
:1049C000170618060906089500240A9412161306FD
:1049D000140605060895092E0394000C11F488238B
:1049E00052F0BB0F40F4BF2B11F460FF04C06F5FA7
:1049F0007F4F8F4F9F4F08950024552704C0080E06
:104A0000591F880F991F009729F076956795B8F37D
:104A10007105B9F7802D952F0895991B79E004C091
:104A2000991F961708F0961B881F7A95C9F78095ED
:104A3000089597FB072E16F4009407D077FD09D050
:104A40000E94332507FC05D03EF4909581959F4F39
:104A50000895709561957F4F0895EE0FFF1F0590A3
:104A6000F491E02D0994AA1BBB1B51E107C0AA1FBA
:104A7000BB1FA617B70710F0A61BB70B881F991FFF
:104A80005A95A9F780959095BC01CD010895F894A9
:024A9000FFCF56
:104A9200BE08AF098C095809240901D0012808145D
:104AA2000A321E404D36224C03FF02C902A70233CE
:104AB200024C0265027E0200010203040506070899
:024AC2000900E9
:106800008800EA44E944E244040005000600070069
:10681000080009000A000B000C000D000E000F001C
:1068200010001100120013001400150016001700CC
:10683000180019001A001B001C001D001E001F007C
:10684000200021002200230024002500260027002C
:10685000280029002A002B002C002D002E002F00DC
:10686000300031003200330034003500360037008C
:10687000380039003A003B003C003D003E003F003C
:1068800040004100420043004400450046004700EC
:10689000480049004A004B004C004D004E004F009C
:1068A000500051005200530054005500560057004C
:1068B000580059005A005B005C005D005E005F00FC
:1068C000600061006200630064006500850067008D
:1068D000680069006A006B006C006D006E006F005C
:1068E0007000710072007300890087008A008B00BD
:1068F000E000E100E200E300F1A1E500E600E700CE
:106900000100010001000100EA4401000100E2442D
:106910000100010001000100460001004A004B0097
:10692000010001004700480001000100E9440100A6
:106930000100010001000100010001003A003B00DC
:106940003C003D003E003F0040004100420043004B
:10695000010035004C0039000100440045005200A0
:1069600049000100010050004F0029004D004E0079
:1069700051000100680069006A006B006C006D0046
:106980006E006F0070007100720073000100010062
:1069900001000100010001000100010001004D00A3
:1069A0004A004E004B0001000100010001000100FF
:1069B00001000100010001000100010001000100CF
:1069C00001000100010001000100010001000100BF
:1069D00001000100010001000100010001000100AF
:1069E0000100010001000100490001000100010057
:1069F000010001000100010001000100010001008F
:00000001FF
